S12301007E012C486561646572203D200420416C6C6F63203D20042020526F6F74203D2079
S10B0120044572726F722004A1
S123012CBDC02186F09702BD02A4BD02C927037E025C7F01287F01297F012A7F012BCE019C
S123014C03BDC009CE012ABDC015BDC021BD0268CE1000864DB710008643B710018646B72A
S123016C10028653B710038602B71004CE0000FF1005CEFFFFFF1007CE5555FF1009CE0045
S123018C01FF102BCE0080FF102DCE0081FF102FCE0088FF1031BD028DBD02C927037E02E9
S12301AC5CCE010DBDC0097C012BCE012ABDC015BD02685FCE1000C18A22066C00085C2077
S12301CCF6BD028DBD02687C012B5FC17D2209BD028D7C012B5C20F3862DBDC0038620BD3D
S12301ECC003CE012ABDC015BDC021BD02C927037E025CCE0117BDC0097C012BCE012ABDAB
S123020CC015BD0268BD028D7C012BBD028D7C012BBD028D7C012BBD028D7C012BBD028DB6
S123022C7C012BBD028D7C012BBD028D7C012BBD028D862DBDC0038620BDC003CE012ABDC3
S123024CC015BDC021BD02C927037E025C7EC000CE0121BDC009BDC0217EC000CE10008C93
S123026C120022056F000820F639CE1000BD02BFBD02D88601B79FD28620B79FD77E02F585
S123028C39CE1000BD02BFBD02D88601B79FD28630B79FD77E030F398604B79FD7BD02BF92
S12302AC86E0B79FD68601B79FD186EFB79FD7BD02BF39B69FD78480810026F739B69FD762
S12302CC840181002704B69FD1394F39B6012BB79FD3B6012AB79FD4B60129B79FD5B6011E
S12302EC28840F8AE0B79FD639BD02BFB69FD784088108260CB69FD0A70008BD02C927E907
S120030C394F39BD02BFB69FD784088108260CA600B79FD008BD02C927E9394F39F1
S9030000FC
